S025000062696E2F64656D6F70726F675F6F6C696D65785F73746D3332653430372E7372656335
S3150800C0001C1D0020E1C4000811C9000811C9000858
S3150800C01011C9000811C9000811C9000811C900088A
S3150800C02011C9000811C9000811C9000811C900087A
S3150800C03011C9000811C9000811C9000801C900087A
S3150800C04011C9000811C9000811C9000811C900085A
S3150800C05011C9000811C9000811C9000811C900084A
S3150800C06011C9000811C9000811C9000811C900083A
S3150800C07011C9000811C9000811C9000811C900082A
S3150800C08011C9000811C9000811C9000811C900081A
S3150800C09011C9000811C9000811C9000811C900080A
S3150800C0A011C9000811C9000811C9000811C90008FA
S3150800C0B011C9000811C9000811C9000811C90008EA
S3150800C0C011C9000811C9000811C9000811C90008DA
S3150800C0D011C9000811C9000811C9000811C90008CA
S3150800C0E011C9000811C9000811C9000811C90008BA
S3150800C0F011C9000811C9000811C9000811C90008AA
S3150800C10011C9000811C9000811C9000811C9000899
S3150800C11011C9000811C9000811C9000811C9000889
S3150800C12011C9000811C9000811C9000811C9000879
S3150800C13011C9000811C9000811C9000811C9000869
S3150800C14011C9000811C9000811C9000811C9000859
S3150800C15011C9000811C9000811C9000811C9000849
S3150800C16011C9000811C9000811C9000811C9000839
S3150800C17011C9000811C9000811C9000811C9000829
S3150800C18011C9000811C90008EE11AA55BFF34F8F4F
S3150800C1904FF46D42CEF20002D16801F4E061042347
S3150800C1A0C0F2FA530B43D360BFF34F8FFEE700BFCD
S3150800C1B010B504464FF4A050C4F2010020214DF6F4
S3150800C1C04D03C0F60003984701280BD14FF4A05041
S3150800C1D0C4F201004DF64503C0F6000398472070E7
S3150800C1E0012010BD002010BD2DE9F04F8DB0202094
S3150800C1F001214DF2CD63C0F60003984704200121C2
S3150800C2004DF2856BC0F6000BD8474FF4006AC4F2AE
S3150800C210020A5046062108224DF28157C0F6000749
S3150800C220B847504607210822B84700258DF81A5006
S3150800C2304FF001088DF81B8002268DF81860402300
S3150800C24005938DF81960504605A94DF2E949C0F6DF
S3150800C2500009C8478DF8186080230593504605A93C
S3150800C260C8474FF461430893ADF82450ADF82650FB
S3150800C270ADF82850ADF82C500C23ADF82A304FF401
S3150800C280A05AC4F2010A504608A94DF24573C0F6F1
S3150800C29000039847504641464DF62903C0F6000369
S3150800C2A0984730464146D8474FF4806AC4F2020A96
S3150800C2B0504605210922B847504606210922B847A3
S3150800C2C0602303938DF810608DF811608DF8125075
S3150800C2D08DF81380504603A9C8474FF0C060414601
S3150800C2E04DF2A963C0F6000398474FF4D040C4F254
S3150800C2F000004DF2C113C0F60003984705A84DF299
S3150800C3001943C0F6000398474FF2FC01C0F6000136
S3150800C3104FF4FA704AF210426E5C4B195F78F319C3
S3150800C32003FB000392FBF3FE03FB1E2EBEF1000F78
S3150800C33006D192FBF3F4631E9BB2B3F5806F03D369
S3150800C3400235242DE8D101E00097019600258DF8E5
S3150800C3501A508DF81B508DF81C508DF81D508DF80D
S3150800C3601E508DF81F508DF816508DF81750019AEB
S3150800C370531E8DF81830009A531E8DF819300CA9E3
S3150800C38021F81C4D4FF4D040C4F200004DF20523AD
S3150800C390C0F6000398470E238DF82A308DF82B50E7
S3150800C3A001238DF82C30ADF82050ADF82250ADF8A9
S3150800C3B02450ADF82650ADF828508DF82D3008A831
S3150800C3C04DF2F123C0F6000398470DB0BDE8F08F93
S3150800C3D000B587B040F2C503C2F200031B78BBB9AB
S3150800C3E040F28000C2F200004CF2B113C0F600031E
S3150800C3F09847012841D140F2C503C2F20003012241
S3150800C4001A7040F2C403C2F2000300221A7034E024
S3150800C41040F2C403C2F2000318782D4B18444CF2BC
S3150800C420B113C0F600039847012826D140F2C40389
S3150800C430C2F200031A780132D2B21A7040F28003AF
S3150800C440C2F200031B78934217D140F2C503C2F229
S3150800C450000300221A7040F28003C2F200035B78E0
S3150800C460FF2B0AD140F28003C2F200039B7823B95E
S3150800C4704CF28D13C0F6000398474FF4D040C4F22F
S3150800C480000000214DF2D143C0F600039847D8B109
S3150800C4904FF4D040C4F20000002101AA4DF23943FE
S3150800C4A0C0F60003984740F26762019B93420BD19E
S3150800C4B09DF80F30FF2B07D19DF8103023B94CF2A9
S3150800C4C08D13C0F60003984707B05DF804FB00BF5C
S3150800C4D08100002008B54CF28D13C0F6000398477A
S3150800C4E010B517498D4640F20002C2F2000240F22A
S3150800C4F01403C2F200039A4210D2131D0F4CE41A19
S3150800C50024F003040434002310464FF22811C0F621
S3150800C51000015A581A500433A342FAD109480A4965
S3150800C5204FF000028842B8BF40F8042BFADB4CF6FD
S3150800C5304D03C0F60003984710BD00BF1700002042
S3150800C5401C1D0020800000201C15002062B67047C4
S3150800C55030B583B0042001214DF28563C0F600038F
S3150800C56098474FF40055009501238DF804300022B2
S3150800C5708DF806208DF8073002238DF805304FF424
S3150800C5800064C4F20204204669464DF2E943C0F647
S3150800C59000039847204629464DF27953C0F6000312
S3150800C5A0984703B030BD00BF10B54CF6F503C0F68A
S3150800C5B000039847044640F2C803C2F200031B680A
S3150800C5C0C31AB3F5FA7F2DD340F2CC03C2F20003A7
S3150800C5D01B788BB940F2CC03C2F2000301221A7011
S3150800C5E04FF40060C4F202004FF400514DF27D533F
S3150800C5F0C0F60003984710E040F2CC03C2F20003ED
S3150800C60000221A704FF40060C4F202004FF4005181
S3150800C6104DF27953C0F60003984740F2C803C2F2B8
S3150800C62000031C6010BD00BF10B54CF6B163C0F620
S3150800C630000398474CF6F504C0F60004A04740F2FC
S3150800C640D403C2F2000300F5FA701860A04740F25E
S3150800C650D003C2F2000300F51C50103018604DF6E6
S3150800C660F523C0F60003984740F6D463C2F20003E8
S3150800C6704FF6A9621A8043F61371598040F6D063C3
S3150800C680C2F200034FF6FF7119800021598040F667
S3150800C690CC63C2F200031A8040F213125A804EF697
S3150800C6A003004DF62933C0F6000398474DF2DD0323
S3150800C6B0C0F60003984710BD08B540F69C63C2F261
S3150800C6C000031B7813F0400F11D113F0020F0ED0A0
S3150800C6D040F6A063C2F200031B681A79FF2A06D146
S3150800C6E05B7923B94CF2D543C0F60003984708BDD9
S3150800C6F010B54DF20113C0F600039847002853D031
S3150800C70040F69062C2F20002108040F6D863C2F288
S3150800C71000039C894FF400604EF62133C0F60003EF
S3150800C720984784421CD101204DF65D33C0F60003BC
S3150800C730984740F69063C2F200031B88A3B34EF6EF
S3150800C740DD53C0F6000398474DF25913C0F60003AF
S3150800C750984740F69063C2F2000300221A8023E04D
S3150800C76040F6D863C2F200039C8940F606004EF6EE
S3150800C7702133C0F600039847844215D14EF69D43EF
S3150800C780C0F60003984740F69063C2F200031B8880
S3150800C79053B14DF25913C0F60003984740F690631B
S3150800C7A0C2F2000300221A804CF6F503C0F6000315
S3150800C7B0984740F2D403C2F200031B6898422BD371
S3150800C7C040F2D402C2F2000203F5FA73136040F68F
S3150800C7D0A463C2F2000340F6A862C2F200021A601D
S3150800C7E002204DF65D33C0F60003984740F6906385
S3150800C7F0C2F200031B887BB14EF6DD53C0F6000378
S3150800C80098474DF25913C0F60003984740F69063CF
S3150800C810C2F2000300221A804CF6F503C0F60003A4
S3150800C820984740F2D003C2F200031B6898420CD323
S3150800C83040F2D002C2F2000203F51C531033136013
S3150800C8404EF64543C0F60003984710BD08B54DF6A9
S3150800C8505903C0F6000398474CF25153C0F600033B
S3150800C86098474CF6AD03C0F6000398474CF24D5373
S3150800C870C0F6000398474CF22963C0F600039847B0
S3150800C8804CF2E913C0F6000398474CF2A956C0F6D5
S3150800C89000064CF2F165C0F600054CF2D134C0F63C
S3150800C8A00004B047A847A047FBE700BF40F21003C3
S3150800C8B0C2F200031A6844F6D353C1F26203A3FB1B
S3150800C8C002129209013A4EF21003CEF200035A60A0
S3150800C8D04FF46D42CEF20002F02182F823100022B6
S3150800C8E09A600721196040F2D803C2F200031A6061
S3150800C8F0704700BF40F2D803C2F2000318687047B9
S3150800C90040F2D803C2F200031A6801321A6070476F
S3150800C910FEE700BF10B54FF0007001214DF2F1643B
S3150800C920C0F60004A0474FF000700021A04710BDD4
S3150800C9300023036043608360C360036143618361CE
S3150800C940C361036243628362C362036343638363AF
S3150800C950C36340220264202242648364C36403657D
S3150800C96043658365C3650366802242668366C3663C
S3150800C970036743678367C3674FF08062C0F8802008
S3150800C9804FF00072C0F884204FF08071C0F888100C
S3150800C9904FF40011C0F88C10C0F89030C0F89430ED
S3150800C9A0C0F89830C0F89C30C0F8A030C0F8A42071
S3150800C9B0C0F8A8304FF40032C0F8AC204FF48072AB
S3150800C9C0C0F8B020C0F8B430C0F8B830704700BF1F
S3150800C9D082B0002301934FF40043C4F202031A699C
S3150800C9E002F01C02890101F4F8610A43C00281B20F
S3150800C9F00A4342F001021A614FF40042C4F20202ED
S3150800CA004FF6FE71C0F20401019B013301931369CD
S3150800CA1013F0010F02D0019B8B42F5D9019A4FF60C
S3150800CA20FF73C0F204039A421FBF4FF40043C4F2D7
S3150800CA300203586980B208BF002002B0704700BFE1
S3150800CA4010B483B0002301934FF40043C4F20203E9
S3150800CA501C6904F01C0444F00304890101F4F8611C
S3150800CA600C43C00281B20C435A611C614FF4004268
S3150800CA70C4F202024FF6FE71C0F20401019B0133B3
S3150800CA800193136913F0010F02D0019B8B42F5D96C
S3150800CA9001984FF6FF73C0F20403C01A18BF0120AD
S3150800CAA003B05DF8044B70472DE9F04186B00446A3
S3150800CAB00D460023059300934FF40043C4F2020386
S3150800CAC01E6926F01C0601A84DF2A953C0F60003FC
S3150800CAD0984702994FF45343CFF6CE630B444EF270
S3150800CAE0BF12C0F2E402934298BF46F008061AD96C
S3150800CAF04FF24013CFF6E9530B4447F63F02C0F214
S3150800CB007D12934298BF46F00C060CD94FF4F243B7
S3150800CB10CFF66C430B444FF4B442C0F26222934200
S3150800CB2088BF46F004064FF40043C4F202031E61B0
S3150800CB30284600214FF400424CF64123C0F6000374
S3150800CB409847002800F020814FF080630593059BE5
S3150800CB502BB1059B013B0593059B002BF9D1236857
S3150800CB60002B6CD04FF001084CF6D116C0F6000623
S3150800CB704FF6FE77C0F20407009B01330093284660
S3150800CB804146B04700F0040083B213B9009BBB428C
S3150800CB90F2D9009A4FF6FF73C0F204039A4208BF0F
S3150800CBA0002000F0F6800021009128464FF48052BC
S3150800CBB04CF64123C0F600039847002800F0E680AB
S3150800CBC04FF001084CF6D116C0F600064FF6FE7770
S3150800CBD0C0F20407009B0133009328464146B0473C
S3150800CBE000F0200080B210B9009BBB42F2D9009A2F
S3150800CBF04FF6FF73C0F204039A4208BF002000F004
S3150800CC00C88000230093284610214CF6D113C0F69D
S3150800CC100003984700F004039BB21BB14FF400636E
S3150800CC20236201E00023236200F002039BB213B1E2
S3150800CC30002363611EE04FF4804363611AE0636971
S3150800CC40226AD20842EA53022846002192B24CF6DA
S3150800CC504123C0F600039847002800F099806FF03A
S3150800CC607F430593059B2BB1059B013B0593059BCC
S3150800CC70002BF9D14FF40043C4F20203196848F2B5
S3150800CC800F12CFF620720A40A06861680843E1686F
S3150800CC9008432169084361690843A1690843E169B2
S3150800CCA00843216A0843616A0843A16A0843E16A9E
S3150800CCB00843216B0843616B01430A431A60E16B21
S3150800CCC0A26B1143226C1143626C1143A26C11438F
S3150800CCD0E26C1143226D1143626D0A435A60A26DDC
S3150800CCE09A60E26DDA609869A16E626E1143E26E2F
S3150800CCF01143226F1143626F11434FF6417202408E
S3150800CD000A43216E42EA01419961E16FA26F0A4323
S3150800CD10DA6103F58053996943F62372CFF6DE028A
S3150800CD200A40D4F88400D4F880100843D4F8881050
S3150800CD300843D4F88C100843D4F890100843D4F864
S3150800CD4094100843D4F898100843D4F89C10084364
S3150800CD50D4F8A01001430A439A61D4F8A410D4F871
S3150800CD60A820114341F40001D4F8AC201143D4F8AB
S3150800CD70B0201143D4F8B8200A43D4F8B41042EAD4
S3150800CD8081021A60012004E0002002E0002000E091
S3150800CD90002006B0BDE8F08140B14FF40043C4F26C
S3150800CDA002031A6842F008021A6070474FF40043FB
S3150800CDB0C4F202031A6822F008021A60704700BF1C
S3150800CDC040B14FF40043C4F202031A6842F0040269
S3150800CDD01A6070474FF40043C4F202031A6822F03F
S3150800CDE004021A60704700BF4FF41043C4F20203EE
S3150800CDF01A6842F001021A60704700BF4FF41043E8
S3150800CE00C4F20203186800F0010070474FF410439B
S3150800CE10C4F202039A6942F480129A61704700BF0D
S3150800CE2040B14FF41043C4F202039A6942F4005227
S3150800CE309A6170474FF41043C4F202039A6922F4C8
S3150800CE4000529A61704700BF40B14FF41043C4F2D4
S3150800CE5002039A6942F002029A6170474FF410433E
S3150800CE60C4F202039A6922F002029A61704700BF6F
S3150800CE7008B501204CF69953C0F6000398474CF6BE
S3150800CE800D63C0F60003984701204CF6C153C0F65F
S3150800CE900003984701204CF62163C0F60003984723
S3150800CEA001204CF64963C0F60003984708BD00BF49
S3150800CEB02DE9F04FB3B04FF0F05001214DF28564E3
S3150800CEC0C0F60004A04747200121A0474FF4804040
S3150800CED001214DF2CD63C0F60003984701204DF2BB
S3150800CEE03973C0F6000398478E23309300278DF8D0
S3150800CEF0C67002268DF8C4608DF8C7708DF8C560B7
S3150800CF00B846C4F20208404630A94DF2E949C0F6CF
S3150800CF100009C847404601210B224DF28154C0F64C
S3150800CF200004A047404631460B22A047404603214D
S3150800CF300B22A047404607210B22A0474FF4006367
S3150800CF4030938DF8C6708DF8C4608DF8C7708DF86B
S3150800CF50C5604FF4C058C4F20208404630A9C84715
S3150800CF6040460B210A46A047322330938DF8C670F7
S3150800CF708DF8C4608DF8C7708DF8C5604FF4006AE7
S3150800CF80C4F2020A504630A9C847504601210B226E
S3150800CF90A047504604210B22A047504605210B22E4
S3150800CFA0A0474FF4C04330938DF8C6708DF8C4601F
S3150800CFB08DF8C7708DF8C560404630A9C847404609
S3150800CFC00D210B22A04740460E210B22A0474CF606
S3150800CFD01513C0F6000398474CF6E953C0F600034C
S3150800CFE098474CF6FD54C0F60004A0470128FCD02B
S3150800CFF001A84CF63113C0F60003984700240194A3
S3150800D00008944FF400730B930C944FF000430F935E
S3150800D010202312931494159416944FF400630993DD
S3150800D0204FF4804306934FF0020B4CF6D117C0F627
S3150800D03000074FF0030A4CF2F109C0F2070941F262
S3150800D0401968C0F22208A6B230465946B84760F3B6
S3150800D0501F4530465146B84760F30F05454518BF8A
S3150800D0604D4502D00134202CEDD101A8A1B24CF6D1
S3150800D070A923C0F60003984740F68063C2F200036E
S3150800D08040F2D072C2F200029A60DB6000221A6097
S3150800D0905A604FF41041C4F202010B6140F280134A
S3150800D0A0C2F2000340F29010C2F2000098601A60C3
S3150800D0B0DB605A6040225A719A884FF4C86060F360
S3150800D0C00C029A808022DA70CB604CF67163C0F647
S3150800D0D00003984733B0BDE8F08F00BF40F2E8037D
S3150800D0E0C2F2000308221A7000225A7027229A7088
S3150800D0F06922DA705B221A7145225A71704700BF9D
S3150800D10038B540F28013C2F20003DB78DB0920D180
S3150800D11040F28014C2F200046588C5F30D0540F696
S3150800D120D860C2F2000040F29011C2F200012A460D
S3150800D1304EF6B573C0F600039847E37843F08003CC
S3150800D140E3704FF41043C4F2020301229A602846A2
S3150800D15038BD002038BD00BF38B540F68063C2F23E
S3150800D1600003DB78DB0900D0FEE740F69063C2F2E5
S3150800D17000031D8840F2D074C2F20004204640F62F
S3150800D180D861C2F200012A464EF6B573C0F600030E
S3150800D190984740F68063C2F200039C6000221A603A
S3150800D1A0102199705A60C5F30B059D80B022DA707C
S3150800D1B04FF41043C4F2020301225A6038BD00BF7F
S3150800D1C010B54FF4C843C4F2000398420CD14FF08F
S3150800D1D0007001214DF21574C0F60004A0474FF007
S3150800D1E000700021A04710BD4FF0806001214DF26C
S3150800D1F01574C0F60004A0474FF080600021A047D0
S3150800D20010BD00BF036823F002030360036843F000
S3150800D21001030360436813F0010F07D14FF6FF734C
S3150800D220426812F0010F01D1013BF9D1436813F0AE
S3150800D230010F5AD08B79012B03680CBF43F080038A
S3150800D24023F080030360CB79012B03680CBF43F0FE
S3150800D250400323F0400303600B7A012B03680CBFDD
S3150800D26043F0200323F0200303604B7A012B036865
S3150800D2700CBF43F0100323F0100303608B7A012BD5
S3150800D28003680CBF43F0080323F008030360CB7A56
S3150800D290012B03680CBF43F0040323F00403036067
S3150800D2A0CA788B789B0743EA02630A7943EA024302
S3150800D2B04A7943EA02520B88013B1343C361036868
S3150800D2C023F001030360436813F0010F07D04FF6FC
S3150800D2D0FF73426812F0010F01D0013BF9D1406893
S3150800D2E080F0010000F0010070470020704700BF81
S3150800D2F070B4837A012199404FF4C843C4F20003FD
S3150800D300D3F8002242F00102C3F80022D3F81C42E7
S3150800D310CA431440C3F81C42037BCBB94FF4C84335
S3150800D320C4F20003D3F80C421440C3F80C42847AC2
S3150800D330C688458845EA0645483443F83450857A10
S3150800D3408688048844EA0644483503EBC5035C60CE
S3150800D350037B012B19D14FF4C843C4F20003D3F859
S3150800D3600C420C43C3F80C42847A0688458845EA81
S3150800D3700645483443F83450857A8688C48844EA92
S3150800D3800644483503EBC5035C60C37A4BB94FF4D2
S3150800D390C843C4F20003D3F804421440C3F8044255
S3150800D3A008E04FF4C843C4F20003D3F804420C4320
S3150800D3B0C3F80442038943B94FF4C843C4F20003CF
S3150800D3C0D3F814422240C3F814220389012B01BF63
S3150800D3D04FF4C843C4F20003D3F814220A4308BF23
S3150800D3E0C3F81422437B012B01BF4FF4C843C4F290
S3150800D3F00003D3F81C22114308BFC3F81C124FF4CC
S3150800D400C843C4F20003D3F8002222F00102C3F88D
S3150800D410002270BC704700BF00238371C37103727A
S3150800D42043728372C3728370C3700323037102232A
S3150800D430437101230380704730B400EB0113D3F81E
S3150800D440B04104F00404E4B2147224B9D3F8B0412C
S3150800D450640D146003E0D3F8B041E4085460D3F8CF
S3150800D460B04104F002045472D3F8B44104F00F0436
S3150800D4709472D3F8B4311B0AD37400EB011303F585
S3150800D480DC74D3F8B851D572D3F8B8512D0A157390
S3150800D490D3F8B8512D0C5573D3F8B8311B0E9373C6
S3150800D4A06368D37363681B0A137463681B0C53742D
S3150800D4B063681B0E937421B9C36843F02003C360E5
S3150800D4C003E0036943F02003036130BC704700BFE3
S3150800D4D019B9C06800F003007047012906BF006942
S3150800D4E000F0030000207047F0B40023012503264E
S3150800D4F005FA03F20C681440944238D107685A00BA
S3150800D50006FA02F4E44327400760076891F804C066
S3150800D5100CFA02FC4CEA070707600F79013FFFB2D5
S3150800D520012F16D887683C40846087684C799440F8
S3150800D5303C43846047689CB205FA04FC27EA0C075A
S3150800D5404760476891F806C00CFA04F4A4B23C4355
S3150800D5504460C7689CB2640006FA04F427EA040427
S3150800D560C460C468CF7907FA02F22243C260013365
S3150800D570102BBDD1F0BC70470183704741837047BB
S3150800D58010B401F007039B00C90800EB8100046A88
S3150800D5900F21994024EA01010162016A9A40114368
S3150800D5A001625DF8044B704710B44FF46053C4F23F
S3150800D5B002039B6803F00C03042B09D0082B0DD03B
S3150800D5C0002B36D14FF41053C0F2F403036035E054
S3150800D5D04FF4D853C0F2B70303602FE04FF46053FB
S3150800D5E0C4F202035C685A6802F03F0214F4800F22
S3150800D5F04FF46053C4F202035B68C3F3881319BF80
S3150800D6004FF4D854C0F2B7044FF41054C0F2F404DF
S3150800D610B4FBF2F101FB03F14FF46053C4F20203C9
S3150800D6205A68C2F3014201325200B1FBF2F30360B9
S3150800D63004E04FF41053C0F2F40303604FF4605251
S3150800D640C4F202029168C1F3031140F20003C2F268
S3150800D6500003595CC9B2046824FA01F14160946870
S3150800D660C4F382241C5DE4B221FA04F4846092684F
S3150800D670C2F342329B5CDBB2D940C1605DF8044B11
S3150800D680704700BF39B14FF46053C4F202031A6BF6
S3150800D6901043186370474FF46053C4F202031A6BC1
S3150800D6A022EA00001863704739B14FF46053C4F298
S3150800D6B002031A6C1043186470474FF46053C4F29F
S3150800D6C002031A6C22EA00001864704739B14FF455
S3150800D6D06053C4F202035A6C1043586470474FF4FF
S3150800D6E06053C4F202035A6C22EA00005864704779
S3150800D6F039B14FF46053C4F202031A691043186132
S3150800D70070474FF46053C4F202031A6922EA000014
S3150800D7101861704739B14FF46053C4F202031A6AAC
S3150800D7201043186270474FF46053C4F202031A6A32
S3150800D73022EA000018627047DC23C4F22723186027
S3150800D740704700BF30B585B004460D46038A23F4FA
S3150800D75040531B041B0CCA8813430382838923F492
S3150800D760B05323F00C031B041B0C0989AA880A432F
S3150800D77069890A4392B213438381838A23F44073E7
S3150800D7801B041B0CAA891343838268464DF2A953CE
S3150800D790C0F6000398474FF4A052C4F201024FF4B2
S3150800D7A08053C4F201039C4218BF94420CBF039AEB
S3150800D7B0029AA3891BB2002B02EB820202EB8202B9
S3150800D7C0BDBF2B685B00B2FBF3F22968A4BF8900D2
S3150800D7D0B2FBF1F248F21F53C5F2EB13A3FB021397
S3150800D7E05B091D01642003FB1023A08900B20028F1
S3150800D7F00BDADB00323348F21F51C5F2EB11A1FBFD
S3150800D8000321C1F3421129430AE01B01323348F2CE
S3150800D8101F51C5F2EB11A1FB0321C1F343112943A3
S3150800D82089B2218105B030BD29B183899BB243F401
S3150800D830005383817047838923F400531B041B0C10
S3150800D840838170478088C0F30800704703881942AF
S3150800D8500CBF00200120704782B04FF46053C4F219
S3150800D86002031A6842F001021A6000229A601968D7
S3150800D87021F0847121F48031196043F21001C2F25B
S3150800D88000415960196821F480211960DA60009214
S3150800D89001921A6842F480321A604FF46052C4F258
S3150800D8A00202136803F400330193009B01330093CB
S3150800D8B0019B1BB9009BB3F5A06FF2D14FF46053DF
S3150800D8C0C4F202031B6813F4003F14BF01230023AC
S3150800D8D00193019B012B46D14FF46053C4F2020316
S3150800D8E01A6C42F080521A644FF4E042C4F2000205
S3150800D8F0116841F4404111609A689A609A6842F446
S3150800D90000429A609A6842F4A0529A6045F20C4224
S3150800D910C0F240725A601A6842F080721A604FF478
S3150800D9206052C4F20202136813F0007FFBD04FF472
S3150800D9307053C4F2020340F205621A604FF4605352
S3150800D940C4F202039A6822F003029A609A6842F0C7
S3150800D95002029A604FF46052C4F20202936803F01E
S3150800D9600C03082BFAD102B0704700BF30B4013A55
S3150800D9708D18A94214D20B461C785A7802EB042259
S3150800D98092B2104480B2824284BF013080B2023320
S3150800D9909D42F1D8CB432B4423F0010302331944AB
S3150800D9A0A94207D10B781B02184480B2834284BF70
S3150800D9B0013080B230BC704770B540F6D864C2F208
S3150800D9C00004667C143E237C06EB0326B6B230447C
S3150800D9D080B204F11A0108224DF66D15C0F600054D
S3150800D9E0A84704F122013246A847034620B1000A97
S3150800D9F040EA032080B270BD4FF6FF7070BD00BFCD
S3150800DA0070B4C4780C44E4B240F69863C2F20003DA
S3150800DA10DC700D0A82782A44D2B29A7046785E7013
S3150800DA200078187095420DD90136F6B240F698631B
S3150800DA30C2F200035E702EB940F69863C2F2000384
S3150800DA4001301870C9B28C4217DA0132D2B240F6E8
S3150800DA509863C2F200039A707AB940F69863C2F2E4
S3150800DA6000035A780132D2B25A7032B940F6986336
S3150800DA70C2F200031A7801321A7070BC704700BFF0
S3150800DA8010B5014640F6A464C2F2000420680830C6
S3150800DA904DF60123C0F600039847226840F69863BE
S3150800DAA0C2F20003197811725978517299789172F5
S3150800DAB0DB78D37210BD00BF08B5002008491422D0
S3150800DAC04DF66D13C0F600039847034620B1000AC9
S3150800DAD040EA032080B208BD4FF6FF7008BD00BFBC
S3150800DAE0E60E002008B506204DF6B913C0F6000369
S3150800DAF0984708BD40F6C863C2F2000300221A80A0
S3150800DB0040F6A863C2F200035A7640F2F003C2F266
S3150800DB10000301221A7040F2E403C2F200034FF434
S3150800DB2080621A80704700BF40F2F003C2F2000319
S3150800DB3000221A7040F6C863C2F200031B882BB98C
S3150800DB4040F6C863C2F200031880704740F2F0033B
S3150800DB50C2F2000301221A70704700BF38B540F6BA
S3150800DB60A463C2F200031C6840F6A063C2F2000375
S3150800DB70AD4A1A6040F69463C2F200031A6003289D
S3150800DB8016D1637E03F00F03032B40F0AE87238A7A
S3150800DB90002B40F0AA8740F69C63C2F200030822D5
S3150800DBA01A704CF2B963C0F60003984700F0CCBD72
S3150800DBB0022840F0A78040F2E003C2F20003DA78B8
S3150800DBC00132D2B2DA70C2B940F2E003C2F20003FF
S3150800DBD09A780132D2B29A707AB940F2E003C2F268
S3150800DBE000035A780132D2B25A7032B940F2E003D1
S3150800DBF0C2F200031A7801321A7040F69063C2F234
S3150800DC00000300221A8041F21A53C2F200031A8056
S3150800DC10637E03F0FD02052A09D1A37E0133DBB238
S3150800DC20A376782B04BF0023637600F05EBF002B33
S3150800DC3000F05B87228A002A52D0A27E511EA17666
S3150800DC40002A40F05287E27E082A05D0591EC9B23A
S3150800DC50012917D8052A15D10023637640F69C6357
S3150800DC60C2F2000380221A704CF2B963C0F60003B0
S3150800DC70984740F6D863C2F20003142283F82F208F
S3150800DC8000F0AABE042A9DBF03219140C9B23021E3
S3150800DC90A1760132E27603F00F03013B072B00F26F
S3150800DCA02487DFE813F06D0208001000D804220765
S3150800DCB0D8042207D80440F6D863C2F2000300222B
S3150800DCC083F82F2063E240F69C63C2F20003042225
S3150800DCD01A704CF2B963C0F60003984700F085BD88
S3150800DCE003F00F03032B40F0008740F69C63C2F253
S3150800DCF0000308221A704CF2B963C0F6000398476D
S3150800DD0000F022BD40F6D863C2F200039B7B452B88
S3150800DD1040F0EB8640F6D863C2F20003197C5A7CC1
S3150800DD2002EB012040F69063C2F200031B8898427A
S3150800DD3000F3DB8684B240F69063C2F200031C80CF
S3150800DD4040F6D863C2F200031B7D13F03F0F40F084
S3150800DD50CC8640F6D863C2F200035B7D002B40F008
S3150800DD60C48640F6D463C2F200031D882DB940F676
S3150800DD70D463C2F200035B88A3B140F6D863C2F24B
S3150800DD800003DB8BAB4240F0B08640F6D862C2F2A5
S3150800DD90000240F6D463C2F20003128C5B889A42F2
S3150800DDA040F0A3864DF6B923C0F6000398474FF610
S3150800DDB0FF73984240F0998640F6D863C2F2000392
S3150800DDC0DB7D062B32D0012B40F08F8640F6D863D8
S3150800DDD0C2F2000393F82230082B40F0868640F6FC
S3150800DDE0D863C2F20003002283F822209A8C4FF6E9
S3150800DDF0F6739A4240F6D863C2F200038CBF093222
S3150800DE0008329A8440F6D863C2F200035A8BDA8342
S3150800DE109A8B1A845D8340F6D462C2F20002528855
S3150800DE209A8300F05BBE00BF0E0F00204DF6E52377
S3150800DE30C0F6000398474FF6FF73984240F05586A0
S3150800DE4040F6A863C2F20003597E81B340F6D86251
S3150800DE50C2F2000240F6A863C2F20003928C9B88C5
S3150800DE609A4224D140F6D862C2F2000240F6A8636C
S3150800DE70C2F20003528CDB889A4218D140F6D86267
S3150800DE80C2F2000240F6A863C2F20003528B1B8856
S3150800DE909A420CD140F6D862C2F2000240F6A86354
S3150800DEA0C2F20003928B5B889A4200F0918140F699
S3150800DEB0D863C2F2000393F82F3003F03F03022B16
S3150800DEC01CD140F6D863C2F200039A8C40F2DC03F8
S3150800DED0C2F200031A8040F2F003C2F200030021E6
S3150800DEE0197040F6C863C2F200031B8893427BD0C0
S3150800DEF040F2F003C2F2000301221A7040F6D8631A
S3150800DF00C2F2000393F82F3013F0040F40F0ED85AA
S3150800DF1040F6D863C2F20003142283F82F2040F695
S3150800DF209062C2F2000228211180502283F82E2026
S3150800DF3093F8295093F82D2083F8292093F8284040
S3150800DF4093F82C2083F8282083F82C4093F8270090
S3150800DF5093F82B2083F8272083F82B0093F82620A4
S3150800DF6040F2F001C2F200010A7093F82A1083F811
S3150800DF70261083F82A20691CC9B283F82D10C1B966
S3150800DF80611CC9B240F6D863C2F2000383F82C10AC
S3150800DF9079B9411CC9B240F6D863C2F2000383F8C6
S3150800DFA02B1031B940F6D863C2F20003013283F868
S3150800DFB02A2040F6D863C2F20003598C40F2DC02EC
S3150800DFC0C2F2000211809A8C5A8499845A8BDA8399
S3150800DFD09A8B1A8440F6D462C2F2000211885983D9
S3150800DFE052889A8300F047BD40F6A863C2F2000340
S3150800DFF05B7E23B1072B40F08C8500F082BD40F68E
S3150800E000A461C2F2000140F6A863C2F200030B60E5
S3150800E010032199761976002199750420D875D97641
S3150800E0209A8040F6D864C2F20004628CDA80628B69
S3150800E0301A80A28B5A800120587640F2E002C2F27A
S3150800E0400002117819735178597391789973D278B7
S3150800E050DA73188294F82920DA7294F828209A72CA
S3150800E06094F827205A7294F826201A724DF68123BE
S3150800E070C0F60003984794F82E3003F0F002502AB1
S3150800E0807ADD1B095C1FA40040F2F103C2F200030B
S3150800E0901A78002340F6D861C2F200015AE0CA187D
S3150800E0A092F8362072B940F2F001C2F200010B7004
S3150800E0B040F2F103C2F200031A7040F6A864C2F2F5
S3150800E0C000045DE0012A02D10133DBB242E0022AF4
S3150800E0D02BD10D1895F83750042D26D140F2F002B1
S3150800E0E0C2F20002137040F2F103C2F200030222E8
S3150800E0F01A7040F6D863C2F20003034493F8382036
S3150800E10093F8393043EA022240F2DC03C2F20003F4
S3150800E1101A8040F20A639A4238BF134640F6A8644A
S3150800E120C2F200046382A3822AE0084490F837000A
S3150800E13070B940F2F001C2F200010B7040F2F1032F
S3150800E140C2F200031A7040F6A864C2F2000417E08F
S3150800E1500344DBB21846A342A1DB40F2F001C2F247
S3150800E16000010B7040F2F103C2F200031A7040F688
S3150800E170A864C2F2000403E040F6A864C2F20004F0
S3150800E18040F6D863C2F20003102283F82F2040F627
S3150800E190D863C2F2000393F82F2042F0020283F8F4
S3150800E1A02F20022283F83620042283F837200622FD
S3150800E1B083F838200A2283F8392040F69062C2F2A2
S3150800E1C000022C211180602283F82E2000F011BC59
S3150800E1D040F6A463C2F2000340F6A862C2F2000247
S3150800E1E01A6040F69C63C2F2000300221A7040F6D9
S3150800E1F0D863C2F2000393F82F3013F0040F11D03E
S3150800E20040F6A863C2F200035A7640F69C63C2F24F
S3150800E210000320221A704CF2B963C0F6000398472F
S3150800E22000F063BC40F6D862C2F2000292F82E00F3
S3150800E2300009800040F2F002C2F200021070143C9D
S3150800E240201A80B240F69062C2F20002108001F0F5
S3150800E2500F01022903D103F03F02122A1DD010B97B
S3150800E26013F0030F19D040F6D861C2F2000140F648
S3150800E270A862C2F20002C98C1289914240F0A183B9
S3150800E28040F6D861C2F2000140F6A862C2F2000266
S3150800E290098D5289914240F0948313F0100F7AD079
S3150800E2A040F6A863C2F20003198A002973D003F165
S3150800E2B00C004DF60123C0F60003984740F6D863D4
S3150800E2C0C2F2000393F82A4040F69863C2F20003AC
S3150800E2D01B78A3425FD140F6D863C2F2000393F8D5
S3150800E2E02B0040F69863C2F200035B78834252D152
S3150800E2F040F6D863C2F2000393F82C1040F69863F0
S3150800E300C2F200039B788B4245D140F6D863C2F22D
S3150800E310000393F82D2040F69863C2F20003DB78D9
S3150800E320934238D140F6A863C2F200031C735873AF
S3150800E3309973DA73DB7E03BB40F6A863C2F2000367
S3150800E340987D197E9A7E891AA1EBD001C9B2CAB204
S3150800E3500844C0B2987512F0800F1CBF4A42D2B268
S3150800E36040F6A863C2F20003D97DA1EB91010A44E5
S3150800E370D2B2DA7502EBD0021A7640F69C63C2F284
S3150800E380000301221A7040F6A863C2F200031A7E3F
S3150800E3909A7600221A8240F6A863C2F200035A7ED1
S3150800E3A002F00F03013B072B00F29F83DFE813F00F
S3150800E3B00800400013016F02C202F7020903540263
S3150800E3C040F69C63C2F200031B7813F0010F00F0BD
S3150800E3D08C8340F6A863C2F2000303225A7640F6FD
S3150800E3E09C62C2F200024021117000221A8240F695
S3150800E3F09063C2F20003188850B140F69C63C2F2DB
S3150800E400000342221A704DF68123C0F6000398478E
S3150800E41041F21A53C2F2000300221A804CF2B96381
S3150800E420C0F60003984740F6A864C2F200048BE1E0
S3150800E43040F69C63C2F200031B7813F0010F00F04C
S3150800E440B78040F6D863C2F2000393F82F3003F082
S3150800E4503F03122B40F0AC8040F6D863C2F20003AB
S3150800E46093F82E3003F0F002502A6DDD1B095C1F6D
S3150800E470A40040F2F103C2F200031A78002340F622
S3150800E480D861C2F2000152E0CA1892F8362052B991
S3150800E49040F2F001C2F200010B7040F2F103C2F241
S3150800E4A000031A7050E0012A02D10133DBB23EE0C4
S3150800E4B0022A2BD10D1895F83750042D26D140F293
S3150800E4C0F002C2F20002137040F2F103C2F2000336
S3150800E4D002221A7040F6D863C2F20003034493F886
S3150800E4E0382093F8393043EA022240F2DC03C2F2BC
S3150800E4F000031A8040F20A639A4228BF1A4640F679
S3150800E500A863C2F200035A829A821DE0084490F872
S3150800E510370050B940F2F001C2F200010B7040F228
S3150800E520F103C2F200031A700EE00344DBB2184688
S3150800E530A342A9DB40F2F001C2F200010B7040F2DF
S3150800E540F103C2F200031A7040F6A864C2F200048E
S3150800E5500323637640F6D863C2F2000393F82620B5
S3150800E560227293F82720627293F82820A27293F8F1
S3150800E5702930E37201204DF68123C0F6000398473F
S3150800E58040F69C63C2F2000342221A7000222282DD
S3150800E59040F69063C2F200031A8041F21A53C2F29F
S3150800E5A000031A804CF2B963C0F600039847CBE023
S3150800E5B040F69C63C2F2000320221A704CF2B9633B
S3150800E5C0C0F60003984740F6A463C2F200031B682E
S3150800E5D000225A7692E440F6D863C2F2000393F812
S3150800E5E02F3013F0010F3ED012F0100F3BD140F63A
S3150800E5F0A863C2F200031B8A002B40F0768240F61D
S3150800E6009064C2F200042088013080B24DF681235E
S3150800E610C0F60003984740F69C63C2F200031A78D6
S3150800E62042F010011970238833B140F69C63C2F298
S3150800E630000342F012021A704CF2B963C0F60003E6
S3150800E640984740F6A864C2F20004012323820823EF
S3150800E65063760023E37640F6D863C2F200031122FC
S3150800E66083F82F20B8E113F0200F18D040F6D863AE
S3150800E670C2F2000393F83400000293F8351040F60E
S3150800E680A063C2F2000340EA01051C682C441C6022
S3150800E69040F69063C2F200031888411B198040F6C1
S3150800E6A09063C2F20003188878B112F0100F0CD1EB
S3150800E6B040F69C63C2F200031A7842F002021A700E
S3150800E6C04DF68123C0F60003984740F6D863C2F298
S3150800E6D0000393F8302093F8313003EB02239BB202
S3150800E6E040F2DC02C2F20002138040F6A862C2F2CF
S3150800E6F00002928A934200D823B940F2DC03C2F2A0
S3150800E70000031A8040F6A863C2F2000340F2DC0256
S3150800E710C2F2000212885A8240F69C63C2F20003D3
S3150800E7201B7813F0030F00F0E08141F21A53C2F28E
S3150800E730000300221A804CF2B963C0F6000398471A
S3150800E74040F6A864C2F2000440F69C63C2F20003D5
S3150800E7501B7813F0200F0ED041F21A53C2F20003B1
S3150800E76000221A80627640F6D863C2F200031422A9
S3150800E77083F82F2030E113F0100F12D041F21A530C
S3150800E780C2F2000300221A8001232382042363763F
S3150800E790E27640F6D863C2F20003112283F82F20EE
S3150800E7A01AE141F21A52C2F200021288DAB113F0E3
S3150800E7B0010F1CBF0023238201D1218A71B9618A06
S3150800E7C08A4282BF41F21A53C2F20003198041F20B
S3150800E7D01A53C2F200031B88238204E041F21A533B
S3150800E7E0C2F2000319800023E37640F6A063C2F262
S3150800E7F0000340F69462C2F2000212681A6041F2FF
S3150800E8001A53C2F200031B887BB1238A6BB140F608
S3150800E8109062C2F200022833138040F6D863C2F22F
S3150800E8200003182283F82F20DCE040F69C63C2F22E
S3150800E83000031B7813F0020F00F0578140F690632F
S3150800E840C2F2000328221A8040F6D863C2F20003F7
S3150800E850102283F82F20C5E040F69C63C2F200031D
S3150800E8601B7813F0010F00F0408140F6A863C2F24E
S3150800E870000300225A7640F69C63C2F20003102277
S3150800E8801A704CF2B963C0F6000398472DE140F6BA
S3150800E8909063C2F20003188820B14DF68123C0F6B2
S3150800E8A00003984740F6D863C2F2000393F82F3066
S3150800E8B013F0010F25D040F69C63C2F200031B78C3
S3150800E8C013F0010F40F6A863C2F200031FBF072228
S3150800E8D05A7600229A7612BF1A8206225A760120A2
S3150800E8E04DF68123C0F60003984740F69C63C2F2B2
S3150800E8F0000310221A704CF2B963C0F60003984759
S3150800E9005FE040F69C63C2F200031B7813F0010F28
S3150800E91008D040F6A863C2F2000305225A76002200
S3150800E9201A82E2E040F69063C2F200031B88002BCD
S3150800E93047D1DAE040F69063C2F20003188820B1A6
S3150800E9404DF68123C0F60003984740F6D863C2F215
S3150800E950000393F82F3013F0010F19D040F6A8637F
S3150800E960C2F2000307225A7600229A7601204DF653
S3150800E9708123C0F60003984740F69C63C2F2000361
S3150800E98010221A704CF2B963C0F60003984718E0D3
S3150800E99040F69063C2F200031B8893B9A5E040F6DF
S3150800E9A09C63C2F200031B7813F0010F00F09D80F0
S3150800E9B040F6A863C2F2000307225A7600229A7626
S3150800E9C093E040F6D863C2F20003102283F82F20A2
S3150800E9D040F6A864C2F2000440F69063C2F200034F
S3150800E9E028221A8040F6D863C2F20003502283F820
S3150800E9F02E20227A40F6D863C2F2000383F82A2032
S3150800EA00627A83F82B20A27A83F82C20E27A83F89C
S3150800EA102D20227B83F82620627B83F82720A27B81
S3150800EA2083F82820E27B83F829200622DA75A28853
S3150800EA305A84E2889A8440F6D462C2F200021188A7
S3150800EA40598352889A832288DA8362881A84637E75
S3150800EA5013F0100F40F6D863C2F200031DBF002260
S3150800EA6083F8312083F83020062202BF83F830204D
S3150800EA700A2283F8312040F6D864C2F20004402303
S3150800EA80A37540F69063C2F200031B881A0A227423
S3150800EA906374002584F8355084F8345065864DF63D
S3150800EAA0E523C0F600039847C04360864523A37351
S3150800EAB0E5736575257540F2DE03C2F200031A8810
S3150800EAC0013292B21A80130AA374E27425834DF6B2
S3150800EAD0B923C0F600039847C043208340F69C63D9
S3150800EAE0C2F2000300221A7038BD40F69063C2F2E3
S3150800EAF0000300221A8040F69C63C2F200031A70D3
S3150800EB0038BD40F2F003C2F2000301211970FFF785
S3150800EB1076BA40F2F003C2F2000301221A70E4E763
S3150800EB20030A43EA002080B2704700BF2DE9F003CC
S3150800EB3040F2F203C2F200034FF0000C83F800C063
S3150800EB4040F2F405C2F200052B4601221F461C8836
S3150800EB50CCB15E88BEB1B0F80080A04513D1448818
S3150800EB60B44210D140F2F203C2F2000383F800C0A7
S3150800EB70086878608B883B8140F25513C2F200031F
S3150800EB801B78BB725AE0541CE4B20C33092C02D031
S3150800EB9094462246DAE72B4600221E461C884CB9C4
S3150800EBA05C883CB940F2F203C2F200031A70082AE4
S3150800EBB036D104E00132D2B20C33082AEDD1002353
S3150800EBC040F25512C2F200021678B0461F46994620
S3150800EBD05FFA83FCAA7AC2EB0804BC42C2BFC2EB46
S3150800EBE00602E146D7B201330C35082BF0D140F2C4
S3150800EBF0F303C2F200031F7040F25413C2F200037B
S3150800EC0083F8009040F2F203C2F2000383F8009002
S3150800EC1040F2F403C2F2000309EB490903EB890643
S3150800EC200268334643F8042B0A6872608A889A8019
S3150800EC3040F25513C2F200031B78B372BDE8F00325
S3150800EC40704700BFF0B440F25513C2F200031E78B5
S3150800EC500136F6B21E7040F2F403C2F20003012236
S3150800EC60002740F2F204C2F20004588819880143CA
S3150800EC7089B259B1997A711A772907DD194601F8C7
S3150800EC80017B5F70013101F8017B0F702270013240
S3150800EC90D2B20C33092AE8D1F0BC704738B540F631
S3150800ECA09063C2F200031B88292B06D840F69063AE
S3150800ECB0C2F2000300221A8038BD40F69063C2F201
S3150800ECC0000300221A8040F6D863C2F200039B8A2A
S3150800ECD0B3F5807F03D0B3F5007F5CD038BD40F62E
S3150800ECE0D862C2F2000240F6D463C2F20003D28CA4
S3150800ECF01B889A426FD140F6D862C2F2000240F6EB
S3150800ED00D463C2F20003128D5B889A4263D1324CF7
S3150800ED10A51F204629464EF62D33C0F60003984710
S3150800ED20A4F11C03002204F8082C022204F8072C7C
S3150800ED3054F8062C626034F8022C228140F2E8026C
S3150800ED40C2F20002106844F8060C928824F8022CD5
S3150800ED5044F8160C24F8122C626844F81C2C2289F4
S3150800ED6024F8182C9A8B62816288A28140F6D462B4
S3150800ED70C2F200021188998352886280082204F838
S3150800ED80102C062204F80F2C40F69063C2F20003FA
S3150800ED902A221A8038BD40F6D862C2F2000240F62E
S3150800EDA0D463C2F20003D28C1B889A4213D140F670
S3150800EDB0D862C2F2000240F6D463C2F20003128D92
S3150800EDC05B889A4207D10449084606394EF62D3320
S3150800EDD0C0F60003984738BDF40E002038B540F653
S3150800EDE0D863C2F20003D98B8AB24FF6FF739A42F0
S3150800EDF015D140F6D863C2F20003188C4FF6FF739C
S3150800EE0098420CD140F6D863C2F200034FF22012A2
S3150800EE10C0F600021068186092889A80B0E040F642
S3150800EE20D463C2F200031B885A4040F6D063C2F28C
S3150800EE3000031B881A4212D140F6D863C2F20003B7
S3150800EE401A8C90B240F6D463C2F200035B8858402D
S3150800EE5040F6D063C2F200035B8818420CD040F239
S3150800EE605813C2F2000340F6CC62C2F200021188BF
S3150800EE70198052885A8005E040F25813C2F20003FE
S3150800EE8019805A8040F25813C2F2000318885D8828
S3150800EE9040F2F403C2F2000300221C46198881429C
S3150800EEA00AD15988A94207D140F2F203C2F20003F7
S3150800EEB01A70082A5BD109E00132D2B20C33082A4B
S3150800EEC0EBD140F2F203C2F200031A7040F6D8649E
S3150800EED0C2F200042046FF2106224FF25D03C0F667
S3150800EEE000039847002384F8203084F8213084F8FA
S3150800EEF0223084F8233084F8243084F8253040F210
S3150800EF00E802C2F200021168C4F80610928862810B
S3150800EF10C4F81610628340F25812C2F20002118831
S3150800EF20E1845288228540F6D462C2F20002118832
S3150800EF30A1835288E283237501226275A373E27363
S3150800EF400822227463740623A3740423E3742273C9
S3150800EF500623637340F6A063C2F2000336341C60CE
S3150800EF6040F69063C2F200032A221A8038BD40F6A2
S3150800EF70D863C2F2000354F8040F1860A2889A8076
S3150800EF8040F6D863C2F2000340F2E802C2F2000279
S3150800EF901168C3F8061092885A8108221A7300224B
S3150800EFA05A7340F69063C2F200031A880E321A802A
S3150800EFB038BD00BF0F2AF0B445D940EA01039B07C4
S3150800EFC045D1A2F110070C4603463F0900EB071688
S3150800EFD0103625681033103443F8105C54F80C5C6E
S3150800EFE043F80C5C54F8085C43F8085C54F8045C75
S3150800EFF043F8045CB342ECD17B1C02F00F0CBCF165
S3150800F000030F4FEA03131944034422D90E461D463B
S3150800F010644656F8047B043C032C45F8047BF8D870
S3150800F020ACF1040402F0030224F00304043423447C
S3150800F030214432B10A4411F8014B914203F8014BBD
S3150800F040F9D1F0BC70470346002AF3D1F9E7034625
S3150800F050F0E76246002AEDD1F3E700BF8307F0B474
S3150800F06048D0541E002A43D0CDB2034602E0002CF5
S3150800F0703ED0144603F8015B13F0030F04F1FF3288
S3150800F080F5D1032C2DD9CDB20F2C45EA052545EA35
S3150800F090054518D9A4F1100703F110061A463F09C9
S3150800F0A006EB07161560103242F80C5C42F8085C4D
S3150800F0B042F8045CB242F5D104F00F040137032C80
S3150800F0C003EB07130DD91E462246043A46F8045B9D
S3150800F0D0032AFAD8221F04F0030422F0030204329A
S3150800F0E013442CB1C9B21C4403F8011BA342FBD13B
S3150800F0F0F0BC704714460346C3E700BF0502060284
S3150800F100060307030803090309040A040B040C048D
S3150800F1100C050D050E050F050F061006100710083D
S30D0800F120FFFFFFFFFFFF0000DF
S3150800F1280000000001020304010203040607080997
S3090800F138007A030A3E
S7050800C00032
